:0200000480007A
:100000006F00C004732F2034930F8000630AFF0336
:10001000930F90006306FF03930FB0006302FF038A
:10002000170F0080130F0FFE63040F0067000F000F
:10003000732F203463540F006F004000136E9E53E3
:10004000171F00002320CFFD6FF09FFF732540F1A5
:100050006310050073251030635805000F00F00F82
:10006000130E100073000000130E00009702000032
:10007000938282F973905230735020307350303035
:1000800073504030970200809382C2F7638C020065
:10009000739052109302B01A739022307323203061
:1000A000E39E62F873500030970200009382420191
:1000B00073901234732540F17300203093001000C8
:1000C00093910000930E1000130E2000639AD12725
:1000D0009300100093911000930E2000130E300037
:1000E0006390D1279300100093917000930E000845
:1000F000130E40006396D125930010009391E00009
:10010000B74E0000130E5000639CD12393001000E3
:100110009391F001B70E0080130E60006392D1231B
:100120009300F0FF93910000930EF0FF130E700008
:100130006398D1219300F0FF93911000930EE0FF9C
:10014000130E8000639ED11F9300F0FF9391700007
:10015000930E00F8130E90006394D11F9300F0FFEC
:100160009391E000B7CEFFFF130EA000639AD11D5C
:100170009300F0FF9391F001B70E0080130EB000D2
:100180006390D11DB720212193801012939100001C
:10019000B72E2121938E1E12130EC0006392D11B25
:1001A000B72021219380101293911000B74E424244
:1001B000938E2E24130ED0006394D119B7202121E1
:1001C0009380101293917000B79E9090938E0E08BA
:1001D000130EE0006396D117B720212193801012EF
:1001E0009391E000B74E4848130EF000639AD11582
:1001F000B7202121938010129391F001B70E008057
:10020000130E0001639ED1139300100093907000B1
:10021000930E0008130E10016394D0131302000014
:1002200093001000939170001383010013021200D9
:1002300093022000E31652FE930E0008130E2001D5
:100240006310D31113020000930010009391E0009B
:100250001300000013830100130212009302200018
:10026000E31452FEB74E0000130E3001631AD30D93
:1002700013020000930010009391F001130000009E
:1002800013000000138301001302120093022000E8
:10029000E31252FEB70E0080130E40016312D30B1F
:1002A00013020000930010009391700013021200DB
:1002B00093022000E31852FE930E0008130E500123
:1002C0006390D10913020000930010001300000096
:1002D0009391E0001302120093022000E31652FEF5
:1002E000B74E0000130E6001639CD105130200009D
:1002F0009300100013000000130000009391F00120
:100300001302120093022000E31452FEB70E008085
:10031000130E70016396D1039310F001930E000049
:10032000130E8001639ED0019300100213904001D0
:10033000930E0000130E90016314D001631CC001E2
:100340000F00F00F63000E00131E1E00136E1E0040
:10035000730000000F00F00F130E10007300000078
:10036000731000C00000000000000000000000004A
:10037000000000000000000000000000000000007D
:040380000000000079
:1010000000000000000000000000000000000000E0
:1010100000000000000000000000000000000000D0
:1010200000000000000000000000000000000000C0
:1010300000000000000000000000000000000000B0
:081040000000000000000000A8
:040000058000200057
:00000001FF
